:100000000EC028C027C026C025C024C023C022C0DF
:1000100021C020C01FC01EC00BC41CC01BC01124A7
:100020001FBECFE5D2E0DEBFCDBF10E0A0E6B0E05E
:10003000E2E3FDE102C005900D92AE39B107D9F7B8
:1000400010E0AEE9B0E001C01D92A13EB107E1F7BA
:10005000A9D66DCED5CFCF93DF93C091DD00D091DF
:10006000DE008091DC00882369F0CE0180969093B9
:10007000DE008093DD008115924021F41092DE00B5
:100080001092DD00E199FECF6091DD007091DE00FD
:1000900040E250E08CEB90E033DE8091DC0088237E
:1000A00041F0E199FECF80E18CBBDFBBCEBBE29A91
:1000B000E19ADF91CF9108951092CA001092CB007F
:1000C0008091C800833011F484E003C0843019F4B7
:1000D00085E08093CA00BFCF813011F020E201C0DB
:1000E00028E18EE790E0ACEBB0E0FC0131913D936C
:1000F0003E2F381B3217D0F3DFCF91E89ABD91E045
:1001000093BF89BD089519BC1ABC13BE0895FBDFC7
:1001100018BA3798F894A89514BE81B5886181BD46
:1001200011BCF89485B7877E806185BF85B7982F0D
:1001300094688B7F806895BF85BF85B7806285BFD7
:100140008895FFCF1092B8009091B800981720F4CE
:1001500090919E009923C1F310929E0008951092F1
:10016000BB001092BA0008951092AA001092A90044
:100170001092A8001092A7001092A6001092A5005D
:1001800008951092E300F0DF66CF1092A300109262
:10019000A2001092A1001092A00008951092B70042
:1001A0001092B5001092B4001092B3001092B200F9
:1001B00008951092E3001092E2008091E1008630F1
:1001C00011F01092E10008958091E300823021F057
:1001D0008091E300843029F48091E3008150809382
:1001E000E3008091E200882361F08091D70090E0E5
:1001F00062E470E014DD845891099093A10080932B
:10020000A000B2CF8091E300811107C09091E2007D
:1002100081E0911103C080E001C081E09091E30092
:10022000933020F49091E200923008F08F5F0895AF
:100230008091CA0090E0880F991FE0916100F091D1
:100240006200E80FF91F808191819093E000809314
:10025000DF000895EDDF8091C800893051F41092DD
:10026000E000E091CA00F0E0E558FF4F8081809304
:10027000DF008091DF00882311F03FDF01C043DF02
:100280008091E000843010F4880F05C0843011F4B0
:1002900087E001C08FE088BB089535DF18BA089564
:1002A00082E12BDF82E04EDF2ECF2091CA0030E0CA
:1002B000220F331FE0916100F0916200E20FF31F03
:1002C000208131812A30310548F0882321F0C2DFB6
:1002D00082E038DFE2CFE1DF82E034CFE1CF1F936D
:1002E000CF93DF93D82FC62F142F19C08C2F05DF83
:1002F000C11102C0D2DF09C0CF3F11F4ABDF05C08E
:10030000CE3F19F481E0D1DF06C0812F1BDFC11180
:1003100002C0A0DF01C0C1DF812F14DFD150D11195
:10032000E5CFDF91CF911F9108951F93CF93DF9376
:100330001F92CDB7DEB7182F82E16983DEDE6981B7
:10034000112339F040E162E181E0C9DF1150D1F7BA
:1003500010C0662321F082E0F5DE19BC08C080E100
:10036000F1DE12E119BD83E0EDDE1150D9F780E135
:10037000E9DE0F90DF91CF911F91C5CECF92DF9232
:10038000EF92FF920F931F93CF93DF93EC01C62E52
:10039000860F911D892B19F460E080E0C6DF55E0DF
:1003A000D52E00E117E26AE0E62EF12CCE01B8016D
:1003B00061DC862F611102C0CD1428F061E0B5DF49
:1003C00081E2C0DECD2CCE01B80154DCEC01C801C5
:1003D000B70150DC8B01DA9449F7DF91CF911F917F
:1003E0000F91FF90EF90DF90CF900895CF93C82F9B
:1003F00080E083DEC7FF08C0C1958BE089BD82E441
:10040000A1DE19BC82E49EDE61E08C2F90E0B6DFB5
:10041000CF9179CE1F93CF93DF9389E06EDE83E097
:1004200091DECBE0C9BD83E08DDED6E1D9BD83E0AE
:1004300089DE11E219BD83E085DE8CE289BD83E0AF
:1004400081DE19BD83E07EDED9BD83E07BDEC9BDE0
:1004500083E078DE89E089BD83E074DE54DE84E0E9
:10046000DF91CF911F916ECE82E147DE81E26ADE9D
:100470008BE089BD81E266DE46CECF938FDE8BE0D6
:100480003CDE80E15FDEC2E1C9BD80E15BDE8BE086
:1004900089BD80E157DEC9BD80E154DEC9BD83E07E
:1004A00051DEC150D9F7CF912ECE8C3221E0920788
:1004B00098F08A3421E0920788F0883621E092078C
:1004C00078F08C3721E0920768F08039914010F481
:1004D00084E0089585E0089580E0089581E008951E
:1004E00082E0089583E008958DDE811110C080912F
:1004F000C800813039F08650833020F08091E100CF
:10050000882329F083E08093B1008093CA00089586
:100510008091CC009091C800993021F0882309F493
:100520003FC001C083E09091CA009093CB009F5FD1
:100530009093CA001092B100943011F41092CA0046
:100540009091CA00981303C01092CA00CDDF5ADE02
:10055000813099F48091CA0090E0880F991FE09152
:100560006100F0916200E80FF91F80819181813074
:10057000924018F01092CA00089544DE823081F44F
:100580008091CA0090E0880F991FE0916100F0917E
:100590006200E80FF91F808191818130914050F70E
:1005A00008958091CC009091C800993021F0882363
:1005B00009F443C001C083E09091CA009093CB003E
:1005C000933011F48093CA009091CA009150909397
:1005D000CA001092B1009F3F51F481508093CA002D
:1005E00083DF05C08091CA0081508093CA000ADE73
:1005F000813081F48091CA0090E0880F991FE091CA
:100600006100F0916200E80FF91F808191818130D3
:10061000924040F7F7DD823081F48091CA0090E08B
:10062000880F991FE0916100F0916200E80FF91FB7
:100630008081918181309140A8F608958091CE000B
:1006400082FD66CFAECF8091CE0082FDAACF60CF73
:10065000CF93C62F40E160E042DE80E173DDC1113F
:1006600044C08091B100811107C04091C800209121
:100670006100309162000AC01092B1008091CB00FD
:100680008093CA0073C051505093CA00433048F061
:10069000473039F0483029F04350423008F066C006
:1006A00010C05091CA005523B9F3E52FF0E0EE0FCA
:1006B000FF1FE20FF31F808191818130924018F774
:1006C000EBCF8091CA0090E0880F991FE091610004
:1006D000F0916200E80FF91F808191818130924092
:1006E00008F444C080E092E03FC044E060E083E072
:1006F000F6DD8091CE0085FD09C04091C8004930EB
:1007000029F0209161003091620004C000DD515059
:100710005093CA00433020F0473011F0483079F44C
:100720005091CA00552359F0E52FF0E0EE0FFF1F5E
:10073000E20FF31F808191818130914040F7435057
:100740004230A0F48091CA0090E0880F991FE09198
:100750006100F0916200E80FF91F80819181813082
:10076000914020F080E091E09183808374DCCF9110
:1007700071CDE82FA49A843010F482E801C08FE88C
:1007800087B987E886B9E23021F0E43011F064E1FE
:1007900001C065E070E080E090E0369A3699FECFC7
:1007A00044B155B1772339F0352F20E0D901A42B7E
:1007B000AD01840F951F7F5F671778F770E05ADAF5
:1007C00037988E2F81508330D0F4CB019695879542
:1007D000969587958093600080E090E0E0916100BD
:1007E000F0916200208D318D40E050E02ADA20E067
:1007F00030E540E050E052DA622F732F17C0E4304A
:10080000A8F08091D600992787FD90958D51914051
:10081000680F791F77FD05C06F3F710509F020F45F
:1008200005C060E070E002C06FEF70E0CB0108959A
:100830001F920F920FB60F9211242F933F934F9355
:100840005F936F937F938F939F93AF93BF93EF9338
:10085000FF938091B8008F5F8093B8008091BB00B8
:100860008F5F8093BB00823459F41092BB0080915B
:10087000BA008F3F29F08091BA008F5F8093BA0051
:100880008091B900882309F4EDC182E072DF909372
:10089000AC008093AB0080916000843108F4B1C05B
:1008A0008091B900823009F0ACC08091CE002091D7
:1008B000AB003091AC0084FF03C08091D00002C037
:1008C0008091D10090E06AE070E0A9D98217930787
:1008D00088F48091A9009091AA009C012F5F3F4F5E
:1008E0003093AA002093A9008234910518F0109249
:1008F000E3003ADC8091CE0084FF46C02091AB003B
:100900003091AC008091D00090E06AE070E087D92F
:1009100082179307C8F12091AB003091AC00809111
:10092000D10090E06AE070E07AD98217930760F511
:100930008091B100833040F58091A7009091A8008C
:100940009C012F5F3F4F3093A8002093A70084386D
:10095000910520F08091E300823058F08091A7004B
:100960009091A8008C3B974078F08091E300823012
:1009700058F08091E300811103C081E08093E3008F
:1009800081E080939F00F0DB2091AB003091AC00C0
:100990008091D10090E06AE070E041D9821793071E
:1009A00080F18091A5009091A6009C012F5F3F4FA0
:1009B0003093A6002093A5008438910520F0809103
:1009C000E300843058F08091A5009091A6008C3B04
:1009D0009740B8F08091E300843098F08091B100A6
:1009E000833020F081E08093E30008C08091E30031
:1009F000833018F483E08093E30082E080939F00CB
:100A0000B3DB809160008431C8F58091B50081111D
:100A100003C081E08093B5008091B200882339F053
:100A20008091B5008F5F8093B5001092B2008091E5
:100A3000B700811105C08091B3008F5F8093B30030
:100A40008091B7008F3F29F08091B7008F5F80932E
:100A5000B7008091B7008B3119F481E08093B40026
:100A60008091B700863319F483E08093B40010922C
:100A7000B6001092AE001092AD0014C01092B700F4
:100A80001092B2008091B6008F3F29F08091B6009D
:100A90008F5F8093B6008091B6008F3018F481E0AC
:100AA0008093B2008091B100833008F1E091CF00D3
:100AB000F0E0EF58FF4F80818823C9F02091AF000C
:100AC0003091B0002F5F3F4F3093B0002093AF00C4
:100AD00090E06AE471E0A3D82817390760F010921B
:100AE000B0001092AF0081E08093B10004C010927A
:100AF000B0001092AF008091E100823021F080912F
:100B0000E1008430B1F48091AD009091AE00019687
:100B10009093AE008093AD008091AD009091AE00B7
:100B20008438910551F48091E10081508093E10077
:100B300004C01092AE001092AD008091C800982FB2
:100B40009650933098F59091B500992379F1909152
:100B50006000943158F19091B900923039F58630A7
:100B600041F48091B400811102C068DD1AC06BDDD0
:100B700018C09091B4008091CD00911109C0982FB8
:100B80009F5F9093CD008D3061F41092CD0009C02D
:100B9000982F91509093CD00811103C08DE08093E8
:100BA000CD0081E080939E0056DAF8DA84E0E1DD42
:100BB0008093A4008091CE0083FF54C08091B9003F
:100BC000823009F04FC08091A4004091D200841778
:100BD00080F48091A2009091A3009C012F5F3F4F71
:100BE0003093A3002093A2008197E0F11092E200DD
:100BF00038C02091A0003091A1002F5F3F4F30936B
:100C0000A1002093A0002091A0003091A1002234E7
:100C1000310520F08091E200882369F02091A00046
:100C20003091A1008091D70090E062E470E0F7D7A6
:100C300028173907B8F02091A400842F90E001967E
:100C400030E0821793073CF081E08093E20083E07C
:100C500080939F0006C084E080939F0082E0809391
:100C6000E20093DAFF91EF91BF91AF919F918F9145
:100C70007F916F915F914F913F912F910F900FBE98
:100C80000F901F901895EF92FF920F931F93CF93A1
:100C9000DF93082F843011F0982F01C092E0E92EE5
:100CA000EA94C0E0D0E041C01092B80010E01EC04D
:100CB00080916000843110F41092B8001091B3005C
:100CC0008091B300813079F48091B400882359F089
:100CD000809160008431E0F381E234DA5FDAFE145F
:100CE00069F110E013C01A3008F019E08091B800E3
:100CF0008436F0F253DA111107C0FE1411F10430FA
:100D000011F1C1E0D0E01FC01F3F59F3CE016AE0EE
:100D100070E085D7EC01C10FD11DFF2029F08BE0D9
:100D2000ECD982E00FDAEFD99F2DF92EFA949111C8
:100D3000BBCF033041F4C851DC4F05C0CFEFD0E04A
:100D400002C0C0E0D0E0CE01DF91CF911F910F91A2
:100D5000FF90EF90089581E2F5D980E0CED9FFD9D8
:100D600004C042E062E181E0BADA8091600084313F
:100D700020F08091BA008823A1F3C5D98091BA00F0
:100D800081110EC0809160008431E0F38091B40045
:100D9000811103C003DA81E0089500DA8FEF08952E
:100DA00080E00895CF93DF9300D01F92CDB7DEB7D8
:100DB00011E08091DC00882309F11AC0E199FECF8F
:100DC00040E250E08CEB90E08BD7E199FECF809130
:100DD000BC008F3F19F01093DC00EBCF8091DD0059
:100DE0009091DE0080969093DE008093DD00E1CF4D
:100DF00081E0BFDC8D3C9105C0F410C06091DD0046
:100E00007091DE00611522E07207C0F2E9C681919F
:100E10008D9330E0EE39F307D1F7EACFDD24D39498
:100E2000853A910520F4D12C02C0A2E0DA2E8FE29F
:100E300087BB18BA8091E300853010F01092E30070
:100E40008091E200833010F01092E200F894A895AF
:100E500081B5886181BD80E481BD789485B7877E46
:100E600085BF8091BB008530E0F382E082DC81E0C9
:100E70008093B900D11001C09CD980916000843169
:100E800008F0A4C096D910E000E023C08091B7001C
:100E90008234F9F41F5F8091C80087FD02C0893059
:100EA00011F40A3091F0173088F4FAD9812F6AE0F2
:100EB000ADD6082F823359F480916000843138F424
:100EC0008091B7008336C0F302C01DE300E01092AA
:100ED000B700809160008431C8F280916000843155
:100EE000E0F35CD90A3009F03FC081E0CCDE90919C
:100EF000C800993019F0893089F405C0893031F083
:100F00001CEF00E07BC69093C90002C08091C9002D
:100F10008093C800D1D89FD87DDA22C081110AC041
:100F20003DD980E20FD983E024DCBFDA60E0FDD94F
:100F30001DEF64C68F3F71F490589093C8008BD812
:100F400069DA8091C80087FF58C609D982E080938A
:100F5000BA0053C6853030F48093C8005BDAACD851
:100F60001BEF4CC68ADA49C6043199F581E08BDE65
:100F7000811109C013D980E2E5D883E0FADB63E090
:100F8000FDD91DEF3DC68430F8F4813061F487E06F
:100F90008093C8008091CA00843010F01092CA007B
:100FA0005AD810E02DC6823011F488E0F1CF80913C
:100FB000C800833018F081E2C5D806C086E080936F
:100FC000E10028DA1CEF1CC658DAFCCF00E010E084
:100FD000AAC1D12C1CEF0E3129F0083219F00233CE
:100FE00009F05AC081E04FDE811144C00E3141F456
:100FF000D5D885E0BEDB882309F4D1C062E0CCC03F
:10100000083201F5CBD814D98091E000882339F05B
:1010100081E298D861E08091E00090E0AFD98091C2
:10102000DF00882369F082E48DD843E06BE083E041
:1010300056D982E487D863E08091DF0090E09ED9A2
:101040001EEF71C1023341F586DE811128C082E4B2
:1010500079D8A4D884E676D8E0916100F091620056
:1010600065E0808D918D8AD984E66CD88091D60018
:10107000BDD9F0CF843078F4080F0F3139F4809166
:10108000C800833030F0F9D900E04DC1093209F4CD
:1010900077C0C0D901C0F1D9023291F401C002E297
:1010A0008091C800863021F08093C90086E002C09C
:1010B0008091C9008093C800CED7ACD91BEF33C153
:1010C0000F3121F0003209F042C021C081E0DBDDA8
:1010D000882309F428C18F3FA1F48091CE0094E0C9
:1010E00089278093CE0082FF0AC08BE006D881E278
:1010F00029D882E189BD81E225D805D813C1B4D9A8
:1011000011C18530C0F581508093CC001DC081E0B5
:10111000BADD882309F407C1982F93509C3F58F1FA
:101120008F3F21F48091CE008C7F0CC0813029F458
:101130008091CE008D7F816005C0823031F4809136
:10114000CE0083608093CE0065D9B6D7ECC0013263
:10115000A1F481E098DD811105C060E08091CF00AD
:10116000E4D883C08F3F19F08A3028F401C080E0B2
:101170008093CF0081C081D9D6C0093209F05DC00B
:10118000EADD81110FC082E4DDD78091CE0083FFBC
:1011900006C062E08091D20090E0F0D866C060E0C6
:1011A00080E0DECF8F3F81F48091CE0098E08927E8
:1011B0008093CE0083FF02C02DD903C060E080E0A1
:1011C000B4D81092E200AEC0813009F0ACC01AD899
:1011D00081115AC08091CE0088608093CE001AD9C8
:1011E000DDD781E2AFD78FE688BB1091A4001F5FE7
:1011F0000FE68091A4001817D8F48091A000909178
:10120000A10001969093A1008093A000819788F39C
:101210001092A1001092A00040D88091A400809369
:10122000D2001091A40017D782E08CD708BBE1CF81
:101230001092A1001092A000DCCF053309F073C01A
:101240008ADD982F82E499837DD7998191110FC00F
:101250008091CE0083FF05C061E08091D7008ED8D9
:1012600003C060E080E061D808D91DEF5CC09F3FFB
:1012700029F48FE08093D700CDD854C0913009F085
:1012800052C0C0D7882321F060E080E04ED84BC028
:10129000C1D882E457D7F090A40045E0F40EE09066
:1012A000CA0083E08093CA00D5D780E09091A40063
:1012B0009F15D8F38F5F2091BB009091BB00291739
:1012C000E1F3853098F3E9D74AD7CF2C90E08091AD
:1012D000A4008F1540F49F5F2091BB008091BB005C
:1012E0002817E1F308C08091A400C81678F7C090D1
:1012F000A400D6D7EBCF953050F38091BA008F5F22
:101300008093D70061E090E039D882E41BD761E098
:101310008C2D90E033D88091CE0088608093CE00F1
:10132000E092CA0098D6802F8A52823018F0043397
:1013300009F078C082E0A7DC7C01009719F581E212
:1013400001D70A3241F48091CE0084FF16C062E0DA
:101350008091D00005C00B3231F462E08091D10061
:1013600090E00CD80DC0043359F48091CE0083FF77
:1013700004C08091D6003AD803C060E080E0D5D7A1
:101380001DEF4FC08F3F910501F50A3249F480915E
:10139000CE0090E189278093CE0084FF0BC033C03C
:1013A0000B3271F48091CE0090E289278093CE00B9
:1013B00085FF04C060E080E0B8D726C055D824C0BF
:1013C000043311F51092D6002AC09C012451310932
:1013D0002734310520F0043311F04FD822C062E0E9
:1013E000C701CCD7B8DC8823E1F00A3241F4E0929F
:1013F000D0008091CE0080618093CE0004C00B327B
:1014000029F4E092D10006D8BCD60BC0043349F4CD
:101410001092D60085E0ADD9E81AE092D600FAD74E
:101420001AD6BCD6033309F05FC083E02CDC0097EA
:1014300069F481E287D6E0916100F091620065E095
:10144000808D918D9BD719D81DEF4CC08F3F910592
:1014500049F4E0916100F091620088EF9AE2918F87
:10146000808F3EC07C01A8EEEA1AA3E0FA0A805BF6
:1014700094408D3B924010F000D834C063E0C70127
:101480007DD769DC882371F184E85CD680E071D96E
:101490005C01B70180E090E020E030E44FE150E0F3
:1014A000D0D3950140E050E0F9D3E0906100F09096
:1014B0006200CA01B90124E630E040E050E0EED31A
:1014C000D70159963C932E93589762337105810545
:1014D000910530F0C901019659969C938E935897C7
:1014E00099D74FD65BD630C00C3371F534DCF82E6B
:1014F000882351F134D680E000D6FBE0EF2E09E1DD
:101500000CC08091BA0080FF02C009BD01C0E9BCD7
:1015100082E018D619BC82E015D680916000843133
:1015200020F08091BA00843060F3EDD50091BA00CC
:1015300081E208D6043040F46DD76CD7BFEFFB12C0
:1015400001C068D78F2DC8D5809160008431E0F349
:1015500025D68091C80087FF1FC080E09091600071
:10156000943130F4FCD5809160008431E0F380E068
:101570009091BA00937089F781110CC082E1BDD5BA
:1015800082E0E0D5C0D585B7806285BF889585B7F4
:101590008F7D85BF81E0E2CF1B3F11F480E107C062
:1015A0001C3F11F481E203C01D3F19F482E4CAD547
:1015B00002C01E3FD9F3D3D5D1101FC09091C800EF
:1015C0009630D9F01E3FC8F48091CE00837081F030
:1015D0002091CA00233089F4813079F4933011F4DA
:1015E00084E002C08091CB008093CA0034D505C04E
:1015F0008091E100863009F05FD58091C800843089
:1016000038F0982F9650933018F08930A9F4F1C231
:10161000E2E0DE1207C0833019F4D092E1000CC082
:101620000DD809C0F1E0DF1207C0833019F4109221
:10163000E10002C008D80FD58091CA00833011F4B0
:101640008093B1008091E100863019F482E08093AC
:10165000E1008091C800843011F41092E100809183
:10166000E100882369F084E06DD542E06EEF85E00B
:1016700036D682E08093E1001092AE001092AD0069
:101680008091E200882361F08091D70090E062E4CD
:1016900070E0C5D2845891099093A1008093A00076
:1016A000D9D582E08093B9008FD510C04EE06FEF9E
:1016B00083E015D682E346D542E36FEF83E00FD691
:1016C0004EE06FEF83E00BD684E83CD58091C800F4
:1016D000863061F334C080919F00882369F0809147
:1016E0009F00813011F460E001C061E080E0B0D77C
:1016F0003BD54BD510929F008091C800873091F464
:10170000A9D584E01FD5C9D580E11CD5A3D584E037
:1017100019D5C3D5E091CD00F0E0ED59FF4F8081A0
:10172000880F10D58091C800883049F4E091CD0031
:10173000F0E0ED59FF4F40816FEF81E0D0D580910F
:10174000C8008750823038F212E0912E0CE1202E32
:1017500083E0782E94E0892E25E0622EC12CDD24D2
:10176000D394A12C42E0B42E56E2352E63E2562EDD
:1017700078E0472E00E014E0E2E3EE2EF12C8091B9
:101780006000843108F420D58091C800813011F0C8
:10179000893099F58091E10081112FC08091B500C9
:1017A000882351F080916000843130F08091B40042
:1017B000811102C043D74ED5809160008431E8F496
:1017C0008091B400813021F43ED744D59092B4008A
:1017D0008091B400833089F49091CE008091CA004A
:1017E00092FF03C0811103C008C0833030F42BD7AF
:1017F00031D59092B4002092B7008091C800823019
:1018000029F48091CC00811104C056C0833009F0C6
:1018100053C08091E10081114FC0809160008431FC
:1018200080F48091B10081110CC0ECD4811109C009
:101830006092B1008091CA008093CB007092CA0080
:1018400009D580916000843170F48091B1008530B9
:1018500051F48091B700803530F08092B1001DD5F1
:1018600082E070D4F7D480916000843158F0809188
:10187000B100853039F41092B1008091CB00809393
:10188000CA00E8D480916000843138F08091B100C2
:10189000843019F47092B100DDD4809160008431FD
:1018A00058F48091B100833039F49092B100809166
:1018B000CB008093CA00CED48091C800843029F038
:1018C0008091E100882309F4F0C08091610090913B
:1018D00062003091CA0020916000243108F097C066
:1018E0002091B700283208F492C06092E100209164
:1018F000B7002E3118F02EE12093B700432F50E0AF
:10190000440F551F480F591F5B834A831092B00044
:101910001092AF008091B500DA012D913C91813099
:10192000E1F42115B4E03B0730F080E09FE6FA01D6
:10193000918380832AC0C901C296B7019BD1620FEF
:10194000731FAA81BB816D937C9361307440E8F072
:10195000EA81FB811183008318C02115310551F004
:10196000C901C296B70186D1261B370BAA81BB815C
:101970002D933C93EA81FB81808191818130944059
:1019800020F0AA81BB810D931C93EA81FB818081A9
:1019900091818C30910518F44092B70007C04697AA
:1019A00018F45092B70002C03092B7002BD48130A7
:1019B00069F4AA81BB818D919C918130924030F075
:1019C000EA81FB81B182A08221E001C020E029836D
:1019D00019D42981823061F4AA81BB818D919C91B7
:1019E0008130914028F0EA81FB81D182C08221E0E0
:1019F000AA81BB818D919C918115944010F4222382
:101A000031F04BD482E09ED325D481E29BD38091E8
:101A1000E1008330E9F41FD31092E1008091C80007
:101A2000833018F49092E10002C0833011F480E01A
:101A30003CD410D48091C800833011F480E182D36B
:101A4000809160008431E0F31092AE001092AD00FE
:101A50008091E100813029F0809160008431F0F4C0
:101A600023C01092E1001092AE001092AD00809160
:101A7000C800843088F780E018D4ECD38091C80087
:101A8000833020F480E15ED380E00FD4E3D380E1A3
:101A900059D3809160008431E0F3DECF8091E10082
:101AA000853011F48092E100D5D3809160008431BB
:101AB000D8F08091B500811104C08091B4008823D2
:101AC00099F06CD38091C800833030F0893021F0D8
:101AD0008091B100833041F495D3823028F4809115
:101AE000E100811101C0B7D280916000843158F0CB
:101AF0008091B100813021F08091B100823019F4E1
:101B000060E080E0A5D580919F00813011F5809143
:101B1000C800833010F41092E1008091B10083304E
:101B200090F48091CA0090E0880F991FE0916100C5
:101B3000F0916200E80FF91F80819181813092401D
:101B400010F49092E30060E082E082D510929F0052
:101B50000BD380919F00823029F58091C80083309B
:101B600010F41092E1008091E30061E0843080F095
:101B70008091CA0090E0880F991FE0916100F09178
:101B80006200E80FF91F808191818130914028F037
:101B900082E05ED58092E30002C080E059D5E4D2B5
:101BA00010929F0080919F00833090F08091C80038
:101BB000833010F41092E10080919F00833011F483
:101BC00060E002C061E083E043D5DFD210929F0065
:101BD00085B7806285BF889585B78F7D85BFCFCD5E
:101BE0001092DE001092DD00EEE7F0E0ACEBB0E02A
:101BF0000EC922E0D21206C013CD1CEFD12CEBC9C6
:101C0000D12C91CB31E0D31217CD14CD002480FD1F
:101C1000060E660F11F08695D1F7802D0895552791
:101C2000002480FF02C0060E571F660F771F611544
:101C3000710521F096958795009799F7952F802D3E
:101C40000895FF27EE27BB27AA2760FF04C0A20F35
:101C5000B31FE41FF51F220F331F441F551F969516
:101C600087957795679589F70097760771F7CF0184
:101C7000BD010895AA1BBB1B51E107C0AA1FBB1FD2
:101C8000A617B70710F0A61BB70B881F991F5A9508
:101C9000A9F780959095BC01CD010895A1E21A2E77
:101CA000AA1BBB1BFD010DC0AA1FBB1FEE1FFF1F00
:101CB000A217B307E407F50720F0A21BB30BE40B50
:101CC000F50B661F771F881F991F1A9469F7609597
:101CD0007095809590959B01AC01BD01CF01089551
:101CE000DC01CB01FC01E199FECF06C0FFBBEEBBDE
:101CF000E09A31960DB20D9241505040B8F70895D8
:101D0000DC01CB0102C02D9105D041505040D8F7E5
:101D10000895262FE199FECF1CBA9FBB8EBB2DBB29
:101D20000FB6F894E29AE19A0FBE01960895F894DE
:021D3000FFCFE3
:101D320064BC007F64503C2D1E140E0A070503028A
:101D42000100020406090C1218243C144BFF140073
:101D520064000002006F0F000A000101000003008E
:0E1D62003F05201D3200F82A000F000000008F
:00000001FF
